:0200000480007A
:100000006F00C004732F2034930F8000630AFF0336
:10001000930F90006306FF03930FB0006302FF038A
:10002000170F0080130F0FFE63040F0067000F000F
:10003000732F203463540F006F004000136E9E53E3
:10004000171F00002320CFFD6FF09FFF732540F1A5
:100050006310050073251030635805000F00F00F82
:10006000130E100073000000130E00009702000032
:10007000938282F973905230735020307350303035
:1000800073504030970200809382C2F7638C020065
:10009000739052109302B01A739022307323203061
:1000A000E39E62F873500030970200009382420191
:1000B00073901234732540F1730020309300400197
:1000C00013016000B3C12002930E3000130E200014
:1000D0006394D10D9300C0FE13016000B3C12002F0
:1000E000930ED0FF130E30006398D10B93004001A4
:1000F0001301A0FFB3C12002930ED0FF130E4000E6
:10010000639CD1099300C0FE1301A0FFB3C120027C
:10011000930E3000130E50006390D109930000003D
:1001200013011000B3C12002930E0000130E6000F3
:100130006394D107930000001301F0FFB3C12002C4
:10014000930E0000130E70006398D1059300000019
:1001500013010000B3C12002930EF0FF130E8000C4
:10016000639CD1039300100013010000B3C120026F
:10017000930EF0FF130E90006390D10393000000E4
:1001800013010000B3C12002930EF0FF130EA00074
:100190006394D101631CC0010F00F00F63000E00D7
:1001A000131E1E00136E1E00730000000F00F00FE0
:1001B000130E100073000000731000C00000000058
:0401C000000000003B
:1010000000000000000000000000000000000000E0
:1010100000000000000000000000000000000000D0
:1010200000000000000000000000000000000000C0
:1010300000000000000000000000000000000000B0
:081040000000000000000000A8
:040000058000200057
:00000001FF
